 
 uniaud16
 
 Start     Length     Name                   Class
 0001:0000 0003cH     _HEADER                DATA
 0001:003c 00614H     _DATA                  DATA
 0001:0650 00bd4H     CONST                  DATA
 0001:1230 00260H     CONST2                 DATA
 0001:1490 00c48H     _BSS                   BSS
 0001:20d8 00004H     _ENDDS                 ENDDS
 0001:20dc 04018H     _HEAP                  ENDDS
 0001:60f4 00002H     _ENDHEAP               ENDDS
 0001:60f8 00000H     _INITDATA              ENDDS
 0001:60f8 00004H     _ENDINITDATA           ENDDS
 0001:60fc 00000H     CONST                  CONST
 0002:0000 0a223H     _TEXT                  CODE
 0002:a224 00000H     RMCODE                 CODE
 0002:a224 00004H     _ENDCS                 CODE
 0002:a228 005acH     _INITTEXT              CODE
 0003:0000 00000H     _TEXT2                 CODE
 
  Address         Publics by Value
 0001:0000       header
 0001:003c       HardwareArray
 0001:017c       fLineTerminate
 0001:017e       dbglevel
 0001:0180       hextab
 0001:019e       APMDD_Name
 0001:01a8       pLincodec
 0001:01ac       usInUseCount
 0001:01ae       usVDDHasHardware
 0001:01b0       IDCVddFuncs
 0001:01be       MaxIDCVddFuncs
 0001:0316       numFreeStreams
 0001:0318       fSetWaveVolume
 0001:03be       MIDISTREAM___usBitNumber
 0001:0426       szCL_DevName
 0001:042e       usCL_HeapSize
 0001:0430       fParamsSpecified
 0001:0432       fVerbose
 0001:0434       fQuietInit
 0001:0436       fFMforMIDI
 0001:0438       fMicMute
 0001:043a       fLineMute
 0001:043c       fCDMute
 0001:045c       szINTEL_ICH
 0001:0466       szALS4000
 0001:0472       szCMEDIA
 0001:047e       szCS4281
 0001:0485       szSBLIVE
 0001:048d       szCS46XX
 0001:0494       szVIA82XX
 0001:049b       szESS1938
 0001:04a6       szVORTEX
 0001:04ad       szES1371
 0001:04b4       szES1370
 0001:04bb       szYAMAHA
 0001:04c2       szMAESTRO
 0001:04ce       szMAESTRO3
 0001:04d7       szALLEGRO
 0001:04df       szALI5451
 0001:04e8       szALI5455
 0001:04f2       szSI7012
 0001:04fd       szNVIDIA
 0001:0504       szAMD
 0001:050c       szTRIDENT
 0001:0514       szNEOMAGIC
 0001:051a       szFM801
 0001:0520       szATIIXP
 0001:0528       szAUDIGYLS
 0001:052f       szBT87X
 0001:0535       szAZX
 0001:053f       FlatDS
 0001:0543       aaulWave
 0001:05c3       aaulAlaw
 0001:05e3       aaulMulaw
 0001:0603       aulSuppSampleRates
 0001:0c30       szSIGMATEL_9721_23
 0001:126e       NumLogicalDevices
 0001:1490       pAudioHWList
 0001:1492       BuildString
 0001:1892       APMDD_Table
 0001:189e       APM_IDC_Entry
 0001:18a2       APM_DS_Reg
 0001:18a4       APM_Enabled
 0001:18a6       APM_Reg_add
 0001:18aa       APM_State
 0001:18ac       APM_Reg_Add
 0001:18b0       Suspend_In_Progress
 0001:18b2       Resume_In_Progress
 0001:18b4       DD_ds
 0001:18b6       APM_Reg_Req
 0001:18c6       fAPMSuspend
 0001:18c8       codec_info
 0001:18f0       pfcodec_info
 0001:18f4       szPddName
 0001:18fd       digit
 0001:190d       current_device
 0001:190f       pWavePlay
 0001:1911       MixerStreamId
 0001:1915       mixcaps
 0001:193d       fRecSrcIOCTL90
 0001:193f       fRecGainIOCTL90
 0001:1941       fPCMVolIOCTL90
 0001:1c44       fInt3BeforeInit
 0001:1c46       fLongNames
 0001:1c54       devCaps
 0001:2094       soundCard
 0001:2095       fNoHardware
 0001:2097       pStreamList
 0001:209d       fNoHWTimer
 0001:209f       pTimerList
 0001:20a1       TIMER___pIRQ
 0001:20a3       TIMER___eTechnology
 0001:20a5       TIMER___usTimerCount
 0001:20a7       TIMER___uInterval_mSec
 0001:20a9       TIMER___uIntervalErr_uSec
 0001:20ac       waveOpened
 0001:20ae       force_closed
 0001:20b0       open_strategy
 0001:20b4       LastSpace
 0001:20b8       ulDeviceSave
 0001:20bc       ulStreamTypeSave
 0001:20c0       ulSysFileNumSave
 0001:20c8       IDCTable
 0001:20d4       Device_Help
 0001:20d8       end_of_data
 0001:20dc       usMemFree
 0001:20de       usUnused
 0001:20e0       pmbFree
 0001:20e2       pmbUsed
 0001:20e4       usnAlloc
 0001:20e6       uscAlloc
 0001:20e8       usnAllocCalls
 0001:20ea       usnFree
 0001:20ec       uscFree
 0001:20ee       usnFreeCalls
 0001:20f0       usnCompact
 0001:20f2       uscTotalHeap
 0001:20f4       acHeap
 0001:60f4       end_of_heap
 0001:60f8       end_of_initdata
 0002:0000       GetHardwareDevice
 0002:0023       SetHardwareType
 0002:0096       GetHardwareType
 0002:00d9       EVENT__Report
 0002:0145       EVENT__GetHandle
 0002:0150       EVENT__GetEventTime
 0002:015b       EVENT__UpdateEvent
 0002:01f0       EVENT__EVENT
 0002:0210       FindEvent
 0002:0237       DecWordToASCII
 0002:02a6       DecLongToASCII
 0002:03d9       HexWordToASCII
 0002:0430       HexLongToASCII
 0002:052f       PrintfOut
 0002:06d7       FMSYNTH__FMSYNTH
 0002:06eb       FMSYNTH__Open
 0002:0755       FMSYNTH__Close
 0002:0759       FMSYNTH__writeByte
 0002:075c       FMSYNTH__readByte
 0002:0760       FMSYNTH__Start
 0002:076f       FMSYNTH__Stop
 0002:0781       FMSYNTH__SetVolume
 0002:07b4       FMSYNTH__dFMSYNTH
 0002:07d4       APM_EVENT
 0002:07ea       APM_COMMAND
 0002:080d       APMEVENT
 0002:08a5       APM_suspend
 0002:08d0       APM_resume
 0002:08fb       apm_resume
 0002:0901       APM_Init
 0002:097a       IDCVddOPENPDD
 0002:0980       IDCVddQUERYPROTOCOL
 0002:0998       IDCVddASSIGNHANDLE
 0002:099d       IDCVddOPENDEVICE
 0002:09ad       IDCVddTRUSTEDOPEN
 0002:09b2       IDCVddCLOSEDEVICE
 0002:09bd       IDCVddGETIOPORTINFO
 0002:09c5       IDCENTRY_VDD_C
 0002:09f9       IoctlAudioInit
 0002:0c1b       IoctlAudioCapability
 0002:0ce0       IoctlAudioControl
 0002:0fc5       IoctlDirectAudio
 0002:1521       StrategyIoctl
 0002:1575       IoctlMixer
 0002:1a65       MixerSetWaveVolume
 0002:1aa9       MixerSetVolume
 0002:1bf3       MixerQueryVolume
 0002:1c8e       MixerQueryProperty
 0002:1c98       MixerSuspend
 0002:1d3a       MixerRestoreState
 0002:1df6       MixerSetProperty
 0002:1f27       MixerNotifyChange
 0002:1f55       HookHandlerIOCTL90
 0002:2002       MixerInit
 0002:23cc       SignatureCheck
 0002:2403       HeapCheck
 0002:247f       npvAllocateBlock
 0002:24fb       malloc
 0002:256b       remove
 0002:2596       compact
 0002:25f3       free
 0002:267c       memfree
 0002:2680       msize
 0002:268f       realloc
 0002:26e6       MIDIAUDIO__DevCaps
 0002:271f       MIDIAUDIO__MIDIAUDIO
 0002:2759       MIDIAUDIO__allNotesOff
 0002:27bd       MIDIAUDIO__Pause
 0002:27bd       MIDIAUDIO__Resume
 0002:27bd       MIDIAUDIO__writeByte
 0002:27c0       MIDIAUDIO__readByte
 0002:27c4       MIDIAUDIO__RTMIDI_OpenReceive
 0002:27c4       MIDIAUDIO__RTMIDI_OpenSend
 0002:27c8       MIDIAUDIO__RTMIDI_CloseReceive
 0002:27c8       MIDIAUDIO__RTMIDI_CloseSend
 0002:27c9       MIDIAUDIO__SetVolume
 0002:27d2       MIDIAUDIO__noteOff
 0002:27ed       MIDIAUDIO__noteOn
 0002:2808       MIDIAUDIO__pitchBend
 0002:2808       MIDIAUDIO__polyphonicPressure
 0002:2826       MIDIAUDIO__controlChange
 0002:2841       MIDIAUDIO__programChange
 0002:285a       MIDIAUDIO__channelPressure
 0002:2870       ddmemmov
 0002:28a1       eMidiByteType
 0002:28be       MIDIMSG__isComplete
 0002:28d5       MIDIMSG__isUnsupported
 0002:28e0       MIDIMSG__addByte
 0002:28f7       MIDIMSG__flush
 0002:2935       MIDIMSG__discardSignature
 0002:2953       MIDIMSG___queryExpectedLength
 0002:29b6       MIDIMSG___queryExpectedSysexLength
 0002:29f9       MIDISTREAM__parse
 0002:2c3c       MIDISTREAM__dispatch
 0002:2eef       MIDISTREAM__CalcDelay
 0002:2f51       MIDISTREAM__Process
 0002:30bc       MIDISTREAM__GetCurrentTime
 0002:30cb       MIDISTREAM__SetCurrentTime
 0002:30ea       MIDISTREAM__Read
 0002:30f0       MIDISTREAM___allNotesOff
 0002:3182       MIDISTREAM__StartStream
 0002:3216       MIDISTREAM__StopStream
 0002:3279       MIDISTREAM__PauseStream
 0002:32d0       MIDISTREAM__ResumeStream
 0002:3362       MIDISTREAM__SetProperty
 0002:33b9       MIDISTREAM__MIDISTREAM
 0002:3478       MIDISTREAM__dMIDISTREAM
 0002:34d1       MPU_401__MPU_401
 0002:3529       MPU_401__Open
 0002:3584       MPU_401__Close
 0002:3588       MPU_401__writeByte
 0002:3590       MPU_401__Reset
 0002:35a3       MPU_401__readByte
 0002:35a7       MPU_401__Start
 0002:35b6       MPU_401__Stop
 0002:35d8       MPU_401__RTMIDI_OpenReceive
 0002:3600       MPU_401__RTMIDI_OpenSend
 0002:3627       MPU_401__RTMIDI_CloseReceive
 0002:3627       MPU_401__RTMIDI_CloseSend
 0002:3631       MPU_401__processIrq
 0002:3696       MPU_401__dMPU_401
 0002:36b5       WTSYNTH__WTSYNTH
 0002:36c9       WTSYNTH__Open
 0002:36f9       WTSYNTH__Close
 0002:371a       WTSYNTH__writeByte
 0002:371d       WTSYNTH__readByte
 0002:3721       WTSYNTH__Start
 0002:3730       WTSYNTH__Stop
 0002:3742       WTSYNTH__SetVolume
 0002:3775       WTSYNTH__dWTSYNTH
 0002:3794       QUEUEHEAD__Head
 0002:379b       QUEUEHEAD__Tail
 0002:37a3       QUEUEHEAD__PushOnHead
 0002:37c0       QUEUEHEAD__PushOnTail
 0002:37e0       QUEUEHEAD__PopHead
 0002:37fe       QUEUEHEAD__PopTail
 0002:3842       QUEUEHEAD__DestroyElement
 0002:3856       QUEUEHEAD__PopElement
 0002:3890       QUEUEHEAD__IsElements
 0002:389f       QUEUEHEAD__QUEUEHEAD
 0002:38ab       RTMIDI___bIsRTMIDIDevice
 0002:38cf       RTMIDI__vConnect
 0002:39b9       RTMIDI__Open
 0002:3a10       RTMIDI__Close
 0002:3a5d       RTMIDI__RecvByte
 0002:3a87       RTMIDI__RecvString
 0002:3ae4       DDCMD_EntryPoint
 0002:3d11       xorstrcmp
 0002:3d34       xorstrncmp
 0002:3d5c       InitializeAudio
 0002:3de3       StrategyInitComplete
 0002:3ec3       StrategyOpen
 0002:3edd       StrategyClose
 0002:3f03       StrategyShutdown
 0002:3f04       StrategyDeinstall
 0002:3f26       StrategyHandler
 0002:3fc6       StrategyHandler2
 0002:4067       STREAM__ReturnBuffer
 0002:40f2       STREAM__ReturnBuffers
 0002:4133       STREAM__ProcessEvents
 0002:4180       STREAM__EnableEvent
 0002:41f8       STREAM__DisableEvent
 0002:423a       STREAM__PauseStreamTime
 0002:4248       STREAM__ResumeStreamTime
 0002:4252       STREAM__Register
 0002:42c2       STREAM__DeRegister
 0002:42d7       STREAM__Write
 0002:4334       STREAM__SetNextEvent
 0002:43aa       STREAM__STREAM
 0002:4451       STREAM__dSTREAM
 0002:44e3       STREAM__SetLooping
 0002:44e4       STREAM__SetProperty
 0002:450f       STREAM__GetProperty
 0002:453a       STREAM__GetCurrentPos
 0002:453a       STREAM__GetCurrentWritePos
 0002:453f       SuspendStreams
 0002:459c       ResumeStreams
 0002:45c7       DestroyStreams
 0002:45e5       FindActiveStream
 0002:4614       FindActiveStream
 0002:4651       FindFirstActiveStream
 0002:467b       FindNextActiveStream
 0002:469a       FindStream_fromFile
 0002:46bc       FindStreamFileId_fromStreamId
 0002:46ea       FindStream
 0002:470c       TIMER___vTimerHook
 0002:473a       TIMER__iCtxHook
 0002:474e       TIMER__TIMER
 0002:47f4       TIMER__vSchedule
 0002:4801       TIMER__ulGetTime
 0002:480e       TIMER__vSetTime
 0002:481b       TIMER__eState
 0002:4823       TIMER___isAnyRunning
 0002:4847       TIMER__Resume
 0002:4847       TIMER__Start
 0002:4847       TIMER___iStart
 0002:48ac       TIMER__Pause
 0002:48ac       TIMER__Stop
 0002:48ac       TIMER___iStop
 0002:48de       TIMER___vPerTickTasks
 0002:4964       TIMER___vStartHWTicks
 0002:4964       TIMER___vStopHWTicks
 0002:4968       IDCENTRY_VDD
 0002:4993       OSSIDC_ENTRY
 0002:49c1       inpd
 0002:49cb       outpd
 0002:49d6       HookHandlerAsm
 0002:49df       HookHandlerIOCTL90Asm
 0002:49e8       WAVEAUDIO__WAVEAUDIO
 0002:4a29       WAVEAUDIO___usfind_matching_sample_rate
 0002:4af8       WAVEAUDIO__QueryDataFlags
 0002:4c3d       WAVEAUDIO__QueryOSSDataFormat
 0002:4eb5       WAVEAUDIO__SetupConversion
 0002:54f8       WAVEAUDIO__QuerySampleFormat
 0002:5630       WAVEAUDIO__FindMatchingSampleRate
 0002:57bc       WAVEAUDIO__DevCaps
 0002:5bbd       WAVEAUDIO__DevCaps
 0002:5bd7       WAVEAUDIO__ConfigDev
 0002:5cc0       WAVEAUDIO__Pause
 0002:5cc0       WAVEAUDIO__Resume
 0002:5cc4       WAVEAUDIO__Start
 0002:5cd9       WAVEAUDIO__Stop
 0002:5cf9       WAVEAUDIO__Prepare
 0002:5d0e       WAVEAUDIO__ConvertPosition
 0002:5d88       WAVEAUDIO__ConvertPositionInvert
 0002:5e20       WAVEAUDIO__ConvertLength
 0002:5e93       WAVEAUDIO__ConvertLengthInvert
 0002:5fe0       ConvertNone
 0002:5fe1       Convert8To8SignChange
 0002:603a       Convert8To16
 0002:6093       Convert8To16SignChange
 0002:60ef       Convert8MonoTo8Stereo
 0002:6148       Convert8MonoTo8StereoSignChange
 0002:61a4       Convert8MonoTo16Stereo
 0002:6207       Convert8MonoTo16StereoSignChange
 0002:625f       Convert8UnsignedTo8UnsignedStereoMono
 0002:62c7       Convert8SignedTo8SignedStereoMono
 0002:632c       Convert8UnsignedTo8SignedStereoMono
 0002:6394       Convert8SignedTo8UnsignedStereoMono
 0002:63fb       Convert8UnsignedTo16UnsignedStereoMono
 0002:6469       Convert8SignedTo16SignedStereoMono
 0002:64dc       Convert8UnsignedTo16SignedStereoMono
 0002:654d       Convert8SignedTo16UnsignedStereoMono
 0002:65c9       Convert16To16SignChange
 0002:6629       Convert16To8
 0002:6684       Convert16To8SignChange
 0002:66e2       Convert16MonoTo16Stereo
 0002:6739       Convert16MonoTo16StereoSignChange
 0002:6793       Convert16MonoTo8Stereo
 0002:67f5       Convert16MonoTo8StereoSignChange
 0002:685a       Convert16UnsignedTo16UnsignedStereoMono
 0002:68ca       Convert16SignedTo16SignedStereoMono
 0002:6937       Convert16UnsignedTo16SignedStereoMono
 0002:69aa       Convert16SignedTo16UnsignedStereoMono
 0002:6a1a       Convert16UnsignedTo8UnsignedStereoMono
 0002:6a87       Convert16UnsignedTo8SignedStereoMono
 0002:6af9       Convert16SignedTo8SignedStereoMono
 0002:6b64       Convert16SignedTo8UnsignedStereoMono
 0002:6bd2       SRateConvert16Stereo
 0002:6c4b       SRateConvert16Mono
 0002:6c4b       SRateConvert8Stereo
 0002:6ccd       SRateConvert8Mono
 0002:6d34       WAVEPLAY__Open
 0002:6ddb       WAVEPLAY__Close
 0002:6de6       WAVEPLAY__ConfigDev
 0002:6f8e       WAVEPLAY__Transfer
 0002:71b0       WAVEPLAY__AddBuffer
 0002:7461       WAVEPLAY__GetPosition
 0002:74d5       WAVEPLAY__GetSpace
 0002:754a       WAVEPLAY__GetHwPtr
 0002:757a       WAVEPLAY__SetVolume
 0002:7594       WAVEPLAY__QueryVolume
 0002:75a9       WAVEPLAY__SetInputSrc
 0002:75b2       WAVEPLAY__dWAVEPLAY
 0002:75d1       WAVEREC__Open
 0002:765d       WAVEREC__Close
 0002:768a       WAVEREC__ConfigDev
 0002:77e7       WAVEREC__Transfer
 0002:7938       WAVEREC__AddBuffer
 0002:7ae9       WAVEREC__GetPosition
 0002:7b55       WAVEREC__GetSpace
 0002:7b99       WAVEREC__GetHwPtr
 0002:7c0c       WAVEREC__SetVolume
 0002:7c2b       WAVEREC__QueryVolume
 0002:7c40       WAVEREC__SetInputSrc
 0002:7c5c       WAVEREC__dWAVEREC
 0002:7c7b       WAVESTREAM___vRealignBuffer
 0002:7d02       WAVESTREAM___vRealignPausedBuffers
 0002:7dee       WAVESTREAM___vUnderrunStop
 0002:7e4b       WAVESTREAM___vUnderrunStart
 0002:7ebf       WAVESTREAM__AddBuffers
 0002:7fe9       WAVESTREAM__AddBuffer
 0002:815e       WAVESTREAM___vReadAudioBuf
 0002:8249       WAVESTREAM__Process
 0002:83fc       WAVESTREAM__Write
 0002:8452       WAVESTREAM__Write
 0002:847a       WAVESTREAM__Read
 0002:84cd       WAVESTREAM__GetCurrentTime
 0002:85a2       WAVESTREAM__GetCurrentPos
 0002:8607       WAVESTREAM__GetCurrentWritePos
 0002:8639       WAVESTREAM__SetCurrentTime
 0002:8646       WAVESTREAM__StartStream
 0002:87dc       WAVESTREAM__StopStream
 0002:88ab       WAVESTREAM__PauseStream
 0002:8965       WAVESTREAM__ResumeStream
 0002:8972       WAVESTREAM__SetProperty
 0002:89dd       WAVESTREAM__GetProperty
 0002:8a0c       WAVESTREAM__WAVESTREAM
 0002:8c6a       WAVESTREAM__dWAVESTREAM
 0002:8d34       HookHandler
 0002:8df8       DWAVESTREAM__Write
 0002:8fad       DWAVESTREAM__ReturnBuffer
 0002:9045       DWAVESTREAM__Register
 0002:90a2       DWAVESTREAM__DeRegister
 0002:90ec       DWAVESTREAM__StartStream
 0002:90ef       DWAVESTREAM__AddBuffers
 0002:922c       DWAVESTREAM__SetProperty
 0002:9288       DWAVESTREAM__GetProperty
 0002:92c4       DWAVESTREAM__DWAVESTREAM
 0002:9345       DWAVESTREAM__dDWAVESTREAM
 0002:9427       OSS16_AttachToPdd
 0002:9473       OSS16_DetachFromPdd
 0002:949b       OSS16_QueryDevCaps
 0002:950e       OSS16_APMResume
 0002:9545       OSS16_APMSuspend
 0002:956f       OSS16_WaveOpen
 0002:95e8       OSS16_WaveClose
 0002:9626       OSS16_WavePrepare
 0002:9660       OSS16_WaveStart
 0002:969a       OSS16_WavePause
 0002:96d5       OSS16_WaveStop
 0002:9710       OSS16_WaveReset
 0002:974b       OSS16_WaveSetFormat
 0002:97a6       OSS16_WaveAddBuffer
 0002:9817       OSS16_WaveGetPos
 0002:9874       OSS16_WaveGetSpace
 0002:98b6       OSS16_WaveGetHwPtr
 0002:98f9       OSS16_WaveGetStatus
 0002:993c       OSS16_WaveSetVolume
 0002:9988       OSS16_MidiOpen
 0002:9a1d       OSS16_MidiWrite
 0002:9a65       OSS16_MidiRead
 0002:9ad5       OSS16_MidiQueryCaps
 0002:9b3d       OSS16_MidiNoteOn
 0002:9b88       OSS16_MidiNoteOff
 0002:9bc9       OSS16_MidiKeyPressure
 0002:9c0b       OSS16_MidiControlChange
 0002:9c4d       OSS16_MidiProgramChange
 0002:9c92       OSS16_MidiChannelPressure
 0002:9cc1       OSS16_MidiPitchBend
 0002:9d03       OSS16_MidiClose
 0002:9d44       OSS16_MixOpen
 0002:9d9a       OSS16_MixClose
 0002:9dca       OSS16_MixSetVolume
 0002:9e1c       OSS16_MixGetVolume
 0002:9e79       OSS16_MixSetProperty
 0002:9ec6       OSS16_MixGetProperty
 0002:9f05       OSS16_MixQueryCaps
 0002:9fce       OSS16_DebugString
 0002:a051       OSSIDC_EntryPoint
 0002:a0d6       _wcpp_2_undefed_cdtor
 0002:a0d8       _wcpp_2_undefined_member_function
 0002:a0da       _wcpp_2_pure_error
 0002:a0dc       _wcpp_2_undef_vfun
 0002:a0de       _wcpp_4_undefed_cdtor
 0002:a0e0       _wcpp_4_undefined_member_function
 0002:a0e2       _wcpp_4_pure_error
 0002:a0e4       _wcpp_4_undef_vfun
 0002:a0e6       new
 0002:a0e9       delete
 0002:a0ec       new
 0002:a0f4       _I4M
 0002:a0f4       _U4M
 0002:a110       _U4D
 0002:a136       _I4D
 0002:a15c       iodelay
 0002:a166       dbgiodelay
 0002:a180       _wcpp_4_dtor_array_store
 0002:a1b0       delete
 0002:a1c0       dtor_the_array
 0002:a204       _wcpp_4_dtor_array
 0002:a224       end_of_text
 0002:a228       StrategyInit
 0002:a4e0       HeapInit
 0002:a51c       memchr
 0002:a536       toupper
 0002:a544       sz2us
 0002:a597       IsWhitespace
 0002:a5ae       SkipWhite
 0002:a5d3       CopyDevicename
 0002:a655       DoParm
 0002:a6cd       ParseParm
 0002:a746       GetParms
 0002:a7b0       WAVEPLAY__WAVEPLAY
 0002:a7c2       WAVEREC__WAVEREC
